S01900006F70656E626C745F73746D3332673037312E7372656300
S315080000000090002069050008490500084B0500080E
S3150800001000000000000000000000000000000000D2
S315080000200000000000000000000000004D05000868
S3150800003000000000000000004F05000851050008F8
S31508000040B9050008B9050008B9050008B90500088A
S31508000050B9050008B9050008B9050008B90500087A
S31508000060B9050008B9050008B9050008B90500086A
S31508000070B9050008B9050008B9050008B90500085A
S31508000080B9050008B9050008B9050008B90500084A
S31508000090B9050008B9050008B9050008B90500083A
S315080000A0B9050008B9050008B9050008B90500082A
S311080000B0B9050008B9050008B9050008E4
S315080000BC10B5064C2378002B07D1054B002B02D024
S315080000CC044800E000BF0123237010BD1000002077
S315080000DC000000004C240008044B10B5002B03D07C
S315080000EC0349044800E000BF10BDC04600000000EC
S315080000FC140000204C240008002243088B4274D3B9
S3150800010C03098B425FD3030A8B4244D3030B8B42FE
S3150800011C28D3030C8B420DD3FF22090212BA030C07
S3150800012C8B4202D31212090265D0030B8B4219D3E8
S3150800013C00E0090AC30B8B4201D3CB03C01A524108
S3150800014C830B8B4201D38B03C01A5241430B8B4250
S3150800015C01D34B03C01A5241030B8B4201D30B0339
S3150800016CC01A5241C30A8B4201D3CB02C01A524160
S3150800017C830A8B4201D38B02C01A5241430A8B4223
S3150800018C01D34B02C01A5241030A8B4201D30B020C
S3150800019CC01A5241CDD2C3098B4201D3CB01C01A26
S315080001AC524183098B4201D38B01C01A5241430930
S315080001BC8B4201D34B01C01A524103098B4201D31E
S315080001CC0B01C01A5241C3088B4201D3CB00C01A8B
S315080001DC524183088B4201D38B00C01A5241430803
S315080001EC8B4201D34B00C01A5241411A00D2014628
S315080001FC524110467047FFE701B5002000F006F89B
S3150800020C02BDC0460029F7D076E770477047C0464E
S3150800021C10B501F083FE10BD10B501F08DFE10BDB2
S3150800022C10B500F0A9FB10BD10B5064B1B699B0455
S3150800023C01D4002010BD00F03FF8FFF7F1FF0120B4
S3150800024CF8E7C0460008005010B5642000F006F820
S3150800025C10BD10B500F008F810BD0000014B188051
S3150800026C7047C0462C00002010B501F009FE0F4B54
S3150800027C1B68984211D30E4B1B78002B0ED10C4BD6
S3150800028C01221A70A023DB051F329A6101F0F8FDD2
S3150800029C084B1B881818054B186010BD044B002218
S315080002AC1A70A023DB0520329A62EFE73000002093
S315080002BC2E0000202C000020A023DB0520229A62A9
S315080002CC7047000070B588B01422002103A802F00C
S315080002DCAFF8144B596B042211435963596B0A40F6
S315080002EC0192019A5A6B012422435A635B6B234091
S315080002FC0093009BA025ED052026AE6280239B016A
S3150800030C029302A9084801F085F802960394002383
S3150800031C04930593069302A9280001F07BF808B00C
S3150800032C70BDC046001002400008005070B590B071
S3150800033C2022002108A802F07BF80C22002104A830
S3150800034C02F076F82C4BD96B802080020143D963D6
S3150800035CDA6B02400192019A5A6B01252A435A63B9
S3150800036C5B6B2B400093009B04230293022403949B
S3150800037C0795A026F60502A9300001F04BF80823CC
S3150800038C029303940024049405940694079502A9F1
S3150800039C300001F03FF80894E1235B0209930A94B4
S315080003AC0B940C940C230D930E940F94134C08A9D0
S315080003BC200001F05DF9A368DB00DB08A360A368E5
S315080003CC0F4A1340A36023680E4A134023606368E0
S315080003DC0D4A13406360A3682A229343A3602368DB
S315080003EC1D432560054BDB699B02FBD5034BDB697B
S315080003FC5B02F7D510B070BD0010024000440040F7
S3150800040CFFFFFFF1FFFFFFDFFFB7FFFF30B5A1B01E
S3150800041C3822002112A802F00BF8102200210EA88F
S3150800042C02F006F83422002101A802F001F8802017
S3150800043C800000F077FA0224129480235B0015934F
S3150800044C00251695C03B179319941A9430221B92C3
S3150800045C1C9380239B021D9380239B041E93C0230D
S3150800046CDB051F9312A800F0E1FA07230E930F94ED
S3150800047C1095119502210EA800F096FD019403958E
S3150800048C01A800F057FE21B030BD10B500F0D0F829
S3150800049CFFF7BCFFFFF716FFFFF748FFFFF7B8FE9D
S315080004ACFFF7BAFEFCE7000000B583B00B4B196CDE
S315080004BC012211431964196C0A400092009ADA6BEE
S315080004CC802149050A43DA63DB6B0B400193019BD8
S315080004DCC020C00000F0CCF803B000BD00100240EC
S315080004EC10B5A024E4052023A3620F4800F044FFAE
S315080004FC200000F041FF0D4BDA6B0D490A40DA6318
S3150800050C5A6B04218A435A635A6B03398A435A63D2
S3150800051C9A6B084802409A63DA6B07480240DA631A
S3150800052C1A6C8A431A6410BD000800500010024069
S3150800053CFFFFFDFFFFFEFFFFFFFFFFEF7047FEE724
S3150800054C7047704710B500F087F810BD024B802233
S3150800055C12059A607047C04600ED00E00D488546C6
S3150800056C002103E00C4B5B58435004310B480C4BF1
S3150800057C42189A42F6D30B4A02E00023136004325F
S3150800058C094B9A42F9D3FFF7E1FF01F02DFFFFF76C
S3150800059C7CFFFEE700900020FC26000800000020E7
S315080005AC10000020100000203C050020FEE700008B
S315080005BC10B5084B01214942D9620022DA62196347
S315080005CC1A6399629A6259625A62FFF789FF002088
S315080005DC10BDC0460010024010B50400114B196836
S315080005EC002901D1012010BDFA208000FFF784FDF7
S315080005FC01000D4B1868FFF77FFD00F077F800280F
S3150800060C0DD1032C01D90120EDE701300022210080
S3150800061C404200F039F8054B1C600020E3E7012046
S3150800062CE1E7C04604000020000000200800002076
S3150800063C10B5084A116880235B000B431360002031
S3150800064CFFF7CAFF041E02D00124200010BDFFF7D5
S3150800065C2BFFFAE700200240034A1368034909688E
S3150800066C5B1813607047C04638050020040000204C
S3150800067C034A136803490B40184310607047C04679
S3150800068C00000140FFF9FFFF70B5002811DB830855
S3150800069C144DC0339B005C5903221040C000FC3239
S315080006AC16008640B44389010A40824022435A51B7
S315080006BC70BDC0B20F230340083B9B0806339B0052
S315080006CC094A944663445D6803242040C000FF220F
S315080006DC14008440A543890111408140294359607F
S315080006ECE6E7C04600E100E000ED00E001380A4B01
S315080006FC98420FD8094A50600948036A1B021B0A1C
S3150800070CC02109060B430362002393600733136069
S3150800071C002070470120FCE7FFFFFF0010E000E017
S3150800072C00ED00E030B5054C61690125294361618E
S3150800073C0260BFF36F8F436030BDC0460020024095
S3150800074C084B5B69002B01DB00207047054B064AFA
S3150800075C9A60064A9A605B69002B01DB0020F4E775
S3150800076C0120F2E70020024023016745AB89EFCD53
S3150800077C064B5969802212060A435A615B69002B9B
S3150800078C01DB012070470020FCE7C0460020024030
S3150800079C70B5050001F07CFB4419174B1B69DB038C
S315080007AC05D501F075FBA042F7D3032070BD124A9C
S315080007BC136912490B401249116192698021C905C6
S315080007CC0A4004D00C488169114381611343002BFC
S315080007DC03D00C4A53600120E8E701F059FB451990
S315080007EC054B1B695B0305D501F052FBA842F7D3F1
S315080007FC0320DBE70020D9E700200240FAC30000FB
S3150800080CFBC3000034000020F8B504000D001600E8
S3150800081C1F00144B1B78012B22D0124B01221A7085
S3150800082C00225A60FA208000FFF7B2FF00280DD18B
S3150800083C012C0FD03100280001F00EFEFA208000A2
S3150800084CFFF7A6FF084A5369A3435361054B0022D9
S3150800085C1A70F8BD32003B002800FFF763FFEDE77E
S3150800086C0220F6E73400002000200240024A5169B3
S3150800087C024B0B43536170470020024004000100F1
S3150800088C044A536904490B40C0001843034B1843E8
S3150800089C506170470020024007FEFFFF020001006E
S315080008AC70B505000E001D4B1B78012B33D01B4B66
S315080008BC01221A7000225A60FA208000FFF768FF9E
S315080008CC002824D12B68042B14D001235B423360F7
S315080008DC6C686B68AA6894466344A34212D92000D4
S315080008ECFFF7CEFFFA208000FFF752FF002808D149
S315080008FC0134EEE7FFF7BAFFFA208000FFF748FF4E
S3150800090C05E03460064A536902218B435361034B55
S3150800091C00221A7070BD0220FCE7C0463400002085
S3150800092C0020024010B5104A136810490B400343C7
S3150800093C136080239B00984201D0002010BD0C4BFD
S3150800094C1A6853009B1858000A49FFF7D5FB013063
S3150800095C054B5B695B0503D5002803D00138F7E71F
S3150800096C0020EBE70320E9E700700040FFF9FFFFE2
S3150800097C0000002040420F0070B501F089FA04000F
S3150800098C254A116880235B000B431360224B1B68B6
S3150800099C5B0506D401F07CFA001B0228F6D9032065
S315080009AC70BD1D4D8023DB016B6001F071FA0400EC
S315080009BC0023AB60184B9B6838221A4207D001F00B
S315080009CC67FA001B154B9842F4D90320E8E7124B3B
S315080009DCC8321A601A6001F05BFA04000E4B1B68E9
S315080009EC9B0106D501F054FA001B0228F6D9032000
S315080009FCD6E7094B80225201DA6000229A61013A45
S31508000A0C1A62074B074A1A60074B1868FFF7E4FD8A
S31508000A1C0028C5D00120C3E7001002408813000047
S31508000A2C000000200024F4000800002070B582B0F5
S31508000A3C041E00D13EE20368DB0739D5C14A91682A
S31508000A4C38230B40D16803220A40102B26D0082BDA
S31508000A5C26D063688022520293427FD0A022D2020B
S31508000A6C934200D181E0B74B1A68B7490A401A601D
S31508000A7C1A68B6490A401A606368002B00D180E0F0
S31508000A8C01F006FA0500AF4B1B689B0310D401F066
S31508000A9CFFF9401B6428F6D903200CE2032AD6D1A9
S31508000AACA84B1B689B0303D56368002B00D104E293
S31508000ABC23689B0731D5A34A936838210B40D16824
S31508000ACC03220A40102B6AD0002B6BD19D4A126860
S31508000ADC520503D5E268002A00D1F0E1994842682C
S31508000AEC9B490A40616909020A434260002B0DD1F1
S31508000AFC036898490B4021690B4303600368DB0ABA
S31508000B0C07221A40944BD340944A1360944B1868A6
S31508000B1CFFF762FD002800D0D3E123681B0700D439
S31508000B2C81E0884B9A6838231340182B73D0A36935
S31508000B3C002B00D191E0834A136E01210B431366F7
S31508000B4C01F0A6F905007F4B1B6E9B076BD401F0D1
S31508000B5C9FF9401B0228F6D90320ACE1794A1168A3
S31508000B6C80235B020B43136086E7764B1968802259
S31508000B7CD2020A431A601968802252020A431A6082
S31508000B8C7AE701F085F905006E4B1B689B038FD538
S31508000B9C01F07EF9401B6428F6D903208BE1022A62
S31508000BAC92D193E7E368002B22D0664A1368694909
S31508000BBC0B4021690B431360116880235B000B43C0
S31508000BCC136001F065F905005E4B1B685B0506D4DE
S31508000BDC01F05EF9401B0228F6D903206BE159494E
S31508000BEC4B685B4A13406269120213434B6094E7E5
S31508000BFC544A13685B490B40136001F049F9050028
S31508000C0C504B1B685B0588D501F042F9401B02283E
S31508000C1CF6D903204FE14B4B1B6E9B0703D5A369F3
S31508000C2C002B00D14FE123685B0700D4A2E0454BAB
S31508000C3C9A6838231340202B22D0424BDB6BDB00FF
S31508000C4C27D4404AD16B802040050143D163D36B2E
S31508000C5C03400193019B01251CE03A4A136E0121BE
S31508000C6C8B43136601F014F90500364B1B6E9B0774
S31508000C7CD9D501F00DF9401B0228F6D903201AE143
S31508000C8C304BDB6D9B0775D5A368002B72D1012001
S31508000C9C11E10025344B1B68DB051FD5A368012B16
S31508000CAC30D0052B34D0274BDA6D01218A43DA650F
S31508000CBCDA6D03318A43DA65A368002B32D001F06A
S31508000CCCE7F806001F4BDB6D9B0751D401F0E0F8E3
S31508000CDC801B264B9842F5D90320ECE0224A116872
S31508000CEC80235B000B43136001F0D2F806001E4B01
S31508000CFC1B68DB05D2D401F0CBF8801B0228F6D989
S31508000D0C0320D8E00F4AD36D01210B43D365D3E7F3
S31508000D1C0C4BDA6D04210A43DA65DA6D03390A439A
S31508000D2CDA65C9E701F0B4F80600064BDB6D9B07DC
S31508000D3C1ED501F0ADF8801B0C4B9842F5D9032053
S31508000D4CB9E0C04600100240FFFFFEFFFFFFFBFFA5
S31508000D5CFF80FFFFFFC7FFFF0024F4000000002000
S31508000D6C08000020FFFEFFFF0070004088130000FB
S31508000D7C012D26D0E369002B00D1A6E0564A9168CE
S31508000D8C38220A40102A63D0022B20D0524B1A68FC
S31508000D9C52490A401A60DA6803218A43DA60DA682B
S31508000DAC4F490A40DA6001F073F804004A4B1B6895
S31508000DBC9B014BD501F06CF8001B0228F6D90320D1
S31508000DCC79E0454AD36B47490B40D363D2E7424A8D
S31508000DDC136842490B40136001F05AF805003E4B64
S31508000DEC1B689B0106D501F053F8401B0228F6D95F
S31508000DFC032060E0384AD3683B491940236A606A85
S31508000E0C0343A06A00020343E06A0343206B0343CF
S31508000E1C606B03430B43D360116880235B040B435D
S31508000E2C1360D16880235B050B43D36001F030F85F
S31508000E3C0400294B1B689B0106D401F029F8001BFA
S31508000E4C0228F6D9032036E0002034E0002032E0F0
S31508000E5C012B3CD0204BDA6803231340216A8B42C2
S31508000E6C01D0012027E070231340616A8B4201D020
S31508000E7C012020E0FE21C9011140A36A1B029942F8
S31508000E8C01D0012017E0F8239B031340E16A8B423B
S31508000E9C01D001200FE0E0231B051340216B8B4288
S31508000EAC01D0012007E0520F5207636B9A4210D00B
S31508000EBC012000E0012002B070BD0120FBE70120F3
S31508000ECCF9E70120F7E70120F5E70020F3E7012011
S31508000EDCF1E70020EFE7C04600100240FFFFFFFED7
S31508000EECFFFFFEEEFFFFFFEF8C80C11110B52B4BF9
S31508000EFC9B6838221A4219D0284B9A683823134013
S31508000F0C082B46D0254B9A6838231340102B18D03B
S31508000F1C224B9A6838231340202B3CD01F4B9A68D7
S31508000F2C38231340182B31D0002009E01B4B1A68C4
S31508000F3CD20A07231340012199401948FFF7DCF818
S31508000F4C10BD164AD1680D3B0B40D2681209072111
S31508000F5C11400131032B0FD11248FFF7CDF80F4B77
S31508000F6CDA68120A7F23134058430C4BD968490F89
S31508000F7C0131FFF7C1F8E3E70948FFF7BDF8074B5E
S31508000F8CDA68120A7F2313405843EEE7FA20C001A9
S31508000F9CD6E70448D4E780200002D1E700100240C7
S31508000FAC0024F40000127A0070B504000D00002825
S31508000FBC00D1AAE0574B1A68072313408B4221D35A
S31508000FCC23689A070ED55B0705D5534A9168E02323
S31508000FDCDB010B439360504A936850490B40A16858
S31508000FEC0B4393602368DB0754D56368012B20D029
S31508000FFC022B3BD0002B3FD1474A126852051CD412
S3150800100C01206AE0434A136807218B432B4313607C
S3150800101C00F03EFF06003F4B1A6807231340AB420D
S3150800102CCED000F035FF801B3D4B9842F3D90320F8
S3150800103C53E0394A1268920369D537498A680720FA
S3150800104C824313438B6000F023FF0600324B9B68E8
S3150800105C38221A406368DB009A421BD000F018FF4E
S3150800106C801B2F4B9842F1D9032036E02A4A126886
S3150800107C9201E2D4012030E0032B05D0264AD26D2A
S3150800108C9207DAD4012028E0234A126E9207D4D4A8
S3150800109C012022E01F4B1A6807231340AB421DD8C8
S315080010AC23685B0706D51C4A93681E490B40E16802
S315080010BC0B439360FFF71AFF174B9A68120A0F2314
S315080010CC13409B00184A9A581F231340D840174BB5
S315080010DC1860174B1868FFF77FFA70BD0D4A13682E
S315080010EC07218B432B43136000F0D2FE0600094BF5
S315080010FC1A6807231340AB42D2D000F0C9FE801BF6
S3150800110C074B9842F3D90320E7E70120E5E70120CE
S3150800111CE3E7C0460020024000100240FFF0FFFF44
S3150800112C88130000FF8FFFFF9C2400080000002096
S3150800113C08000020F0B583B0040003689B0360D553
S3150800114C804BDB6BDB001ED47E4AD16B80204005BE
S3150800115C0143D163D36B03400193019B01267A4A61
S3150800116C116880235B000B43136000F091FE0500A9
S3150800117C754B1B68DB0508D400F08AFE401B022859
S3150800118CF6D9032502E00026E9E70025002D21D132
S3150800119C6C4BDB6DC0229200134010D0226B9A4226
S315080011AC0DD0684AD36D69490B40D06D8021490230
S315080011BC0143D165D16D66480140D165D365DB071E
S315080011CC10D4002D06D15F4AD36D60490B40216BB4
S315080011DC0B43D365012E15D15A4AD36B5D490B4087
S315080011ECD3630FE000F054FE0700564BDB6D9B07EC
S315080011FCE7D400F04DFEC01B574B9842F5D9032592
S3150800120CDFE700252368DB0706D54E4A536D032115
S3150800121C8B4361680B43536523689B0706D5494A7C
S3150800122C536D0C218B43A1680B43536523689B06AE
S3150800123C06D5444A536D49490B40E1680B4353653F
S3150800124C23689B0506D53F4A536D45490B40A16952
S3150800125C0B43536523685B0506D53A4A536D4149DA
S3150800126C0B40E1690B43536523685B0606D5354A83
S3150800127C536D3D490B4021690B43536523685B0449
S3150800128C0BD5304A536D9B009B08216A0B4353655B
S3150800129C8023DB05226A9A4239D023681B0306D5BC
S315080012AC284A536D40218B43616A0B435365236867
S315080012BC9B020BD5234A536D2C490B40A16A0B4351
S315080012CC53658023DB03A26A9A4227D023685B0204
S315080012DC0BD51C4A536D26490B40E16A0B435365E3
S315080012EC80235B04E26A9A421FD023681B050BD540
S315080012FC144A536D1F490B4061690B435365626968
S3150800130C8023DB019A4215D0280003B0F0BD0D4AA4
S3150800131CD16880235B020B43D360BEE7094AD168C8
S3150800132C80235B040B43D360D0E7064AD1680B4392
S3150800133CD360DAE7034AD16880235B020B43D36098
S3150800134CE2E7C0460010024000700040FFFCFFFFB9
S3150800135CFFFFFEFFFFFFFFEF88130000FFF3FFFF01
S3150800136CFFFFF3FFFFFFCFFFFFCFFFFFFFFFBFFF1F
S3150800137CFFFFFFFEFF3FFFFFA023DB0598420DD0C2
S3150800138C1F4B984214D01F4B98421BD01E4B9842A9
S3150800139C22D01E4B984229D0012008E01C4B5A6AD1
S315080013AC01210A435A625A6A8A435A6200207047D4
S315080013BC174B5A6A02210A435A625A6A8A435A6274
S315080013CC0020F4E7124B5A6A04210A435A625A6AF5
S315080013DC8A435A620020EAE70D4B5A6A08210A43E7
S315080013EC5A625A6A8A435A620020E0E7084B5A6ADC
S315080013FC20210A435A625A6A8A435A620020D6E75F
S3150800140C0004005000080050000C00500014005056
S3150800141C00100240F0B5002209E0C66834400E6997
S3150800142C6E433443C4604C68022C1ED001320B68E0
S3150800143C1C00D44034D0012494402340F6D00668CE
S3150800144C1D005D436C006419E44326404F686F43E6
S3150800145C3E4306604E68013E012EDED8866826405D
S3150800146C8F686F433E438660D7E7FF2B0AD8046A1A
S3150800147C5D436B431D01ED1AAC434D696B43234326
S3150800148C0362D3E7456A1B0A1C005C435C4363434F
S3150800149C1C01E41AA5434C6963432B434362C5E715
S315080014AC4A68013A012A01D90020F0BDC968426888
S315080014BC9A434B4313434360F6E70000054B9A687F
S315080014CC120A0F2313409B00034A9A581F231340F2
S315080014DCD8407047001002409C240008054B9A68B7
S315080014EC120B072313409B00034A9A581F231340D9
S315080014FCD840704700100240DC24000810B50E4B8B
S3150800150CDA6803231340032B01D00C4A00E00C4A7B
S3150800151C094CE3681B0A7F2018405043E3681B09F3
S3150800152C072119400131FEF7E7FDE168490F013142
S3150800153CFEF7E2FD10BDC046001002400024F40080
S3150800154C00127A0010B50C4B9A6838231340082BF6
S3150800155C0FD0102B02D1FFF7D1FF10BD064B1A681E
S3150800156CD20A07231340012199400448FEF7C4FD0B
S3150800157CF3E70348F1E7C046001002400024F400E4
S3150800158C00127A0010B50400FFF7DCFF2060FFF7A5
S3150800159C95FF6060FFF7A2FFA06010BD10B5032889
S315080015AC03D00C2827D0002010BD294B5B6D0340B7
S315080015BC00041843274B98420FD0274B984214D057
S315080015CC264B984206D0FFF7BDFFFFF777FFFFF7CC
S315080015DC85FFE9E7FFF7B6FFE6E71D4B1B685B05DA
S315080015EC01D40020E0E71E48DEE7194BDB6D9B07AC
S315080015FC25D40020D8E7164B5B6D0340000418432E
S3150800160C184B98420FD0184B984212D0174B984249
S3150800161C06D0FFF797FFFFF751FFFFF75FFFC3E70A
S3150800162CFFF790FFC0E70A4B1B685B050AD400203E
S3150800163CBAE7074BDB6D9B0706D40020B4E780207E
S3150800164C0002B1E70648AFE780200002ACE7C046C7
S3150800165C001002400200030003000300010003000F
S3150800166C0024F40008000C000C000C0004000C000C
S3150800167C70B584B004000D000368DB0700D579E06B
S3150800168C03683D4A1A408B6809690B4369690B4321
S3150800169CE9690B43134303604368384A1340EA6805
S315080016AC134343608368364A1340AA69134383601D
S315080016BC344B984213D0344B98421AD0334B984239
S315080016CC1BD0334B98421DD001202B68E26A0F21A0
S315080016DC8A431B041B0C1343E36204B070BD03203E
S315080016ECFFF75CFF002841D06E68002E0FD1012051
S315080016FCEBE70C20FFF752FFF4E701A8FFF742FFD0
S3150800170C0398EFE701A8FFF73DFF0398EAE72B6874
S3150800171CEA690B2B2CD8802109028A4210D0FF22A9
S3150800172C13409B001B4A9958FEF7E6FC7308C01831
S3150800173C3100FEF7E1FC0004000CE0600020C4E771
S3150800174CFF2213409B00134A9958FEF7D5FC40001C
S3150800175C7308C0183100FEF7CFFC0F4B0340400846
S3150800176C072210400343E3600020AEE70120ACE7F4
S3150800177C0020AAE70120B0E7F369FFEFFFCFFFFFD0
S3150800178CFFFCFFFF003801400044004000480040C1
S3150800179C004C0040FC240008F0FF000072B67047AD
S315080017AC62B6704710B5FFF7F9FF10BD10B500F01B
S315080017BC77FA002800D110BDFEF736FD0028FAD0BE
S315080017CC00F0E8FBFEF7F4FE00F030FB00F06CFAD4
S315080017DC054B1840054B986000F066FA4468FFF70D
S315080017ECDFFFA047E7E7C04680FFFF1F00ED00E0DC
S315080017FC70B508E04D1C461C0B78037000F0FDFB19
S3150800180C300029002200541EA4B2002AF2D170BD61
S3150800181C70B50500002401E00134E4B20D2C15D88E
S3150800182C00F0EBFB63001B199A00094BD358AB422B
S3150800183CF2D8620012199000054A121852689B18C1
S3150800184CAB42E9D9024B1B18187A00E0FF2070BD91
S3150800185C2C25000870B5050000240D2C10D800F0B6
S3150800186CCCFB63001B199A00074B9B181B7AAB42DF
S3150800187C02D00134E4B2F0E71300034A985870BD5D
S3150800188C01204042FBE7C0462C25000870B5050030
S3150800189C00240D2C10D800F0B0FB63001B199A001D
S315080018AC064B9B181B7AAB4202D00134E4B2F0E724
S315080018BC024B9B18586870BD0020FCE72C250008C5
S315080018CC10B5CB0509D103688B4208D002C080221B
S315080018DC9200FFF78DFF012000E0002010BD0120CB
S315080018ECFCE7F0B5C64600B580460068FFF790FFE2
S315080018FCFF2828D0FEF724FF002500E001353F2DF0
S3150800190C18D8EB0042461268D41843445E689F68A0
S3150800191C00F073FB32003B0021000120FEF774FF38
S3150800192C002809D122686368B24201D1BB42E5D0CE
S3150800193C002402E0012400E00024FEF719FF200031
S3150800194C04BC9046F0BD0024F9E7000070B505000C
S3150800195C0E000F4B984214D00E4B99420BD10C4CDF
S3150800196C2500002C05D031002800FFF7A9FF002818
S3150800197C0CD0200070BDFFF7B4FF012804D000245A
S3150800198CEFE7054C2500ECE72C00EAE70024F0E726
S3150800199C50020020002800084C000020F8B5CE465E
S315080019AC474680B505000C0016001F004B0A5B0263
S315080019BC9846036801330CD02B68434510D1012394
S315080019CC99464B46012B14D048460CBC9046994672
S315080019DCF8BD4146FFF774FF81460028F1D0EBE7C6
S315080019EC41462800FFF7B2FF051E1FD00123994672
S315080019FCE7E72B68E41A2C19043406E033782370CD
S31508001A0C01340136013F002FDED000F0F6FA2B1D0B
S31508001A1CE31A094A9342F1D98021890041442800E6
S31508001A2CFFF794FF051E04D0041DE7E7002399462B
S31508001A3CCAE700239946C7E7FF010000F0B587B04F
S31508001A4C0C0000230593884205D804283BD9122993
S31508001A5C3BD8012600E00026012E02D0300007B044
S31508001A6CF0BDFFF7F7FE07002000FFF7F3FE0500B1
S31508001A7C2000FFF70BFF2D18013DED1B0135ED0A74
S31508001A8CADB202230293F8231B069C466744FF0A51
S31508001A9C039701230493FEF753FE0024AC420FD29E
S31508001AAC00F0ABFA05A902A8FEF7FAFE002806D143
S31508001ABC039B0193013303930134A4B2EEE700268A
S31508001ACCFEF756FECAE70026C8E70026C6E700005A
S31508001ADC01235B42024A1360024A13607047C046F0
S31508001AEC4C0000205002002070B504000E001500B2
S31508001AFC4A1E134B1B1A9A4201D9002070BDFFF7D8
S31508001B0C87FEFF2818D030190138FFF781FEFF2809
S31508001B1C14D0630A5B020B4A934206D033002A00A0
S31508001B2C21000948FFF73AFFE8E733002A002100AD
S31508001B3C0648FFF733FFE1E70020DFE70020DDE783
S31508001B4CFFFF0108002800084C0000205002002066
S31508001B5C70B505000C004A1E0F4B1B1A9A4205D984
S31508001B6CFF21FF260020012812D070BDFFF750FE7A
S31508001B7C060060190138FFF74BFE0100FF2E03D053
S31508001B8CFF2803D00120EEE70020ECE70020EAE767
S31508001B9C3000FFF753FFE8E7FFFF010800B583B0F5
S31508001BAC104B1B6801331BD00E4A536891688C4640
S31508001BBC6344D1688C46634411698C466344516905
S31508001BCC8C46634491698C466344D2699B185B4284
S31508001BDC019301AA04210448FFF786FF03B000BD50
S31508001BEC0120FBE750020020BC2800080E4B1A689F
S31508001BFC0E4B1B68D2180E4B1B689A180D4B1B689C
S31508001C0C9B180D4A1268D3180C4A1268D2180C4B3A
S31508001C1C1B689A180B4B1B689B18002B01D00020CD
S31508001C2C70470120FCE7C046002800080428000875
S31508001C3C082800080C280008102800081428000892
S31508001C4C18280008BC28000810B50B4B1B68013374
S31508001C5C0AD10A4B1B6801330CD00848FFF741FE22
S31508001C6C002808D0012006E00348FFF73AFE0028B2
S31508001C7CEFD100E0012010BD500200204C000020DE
S31508001C8C004870470028000810B5FFF721FF10BD63
S31508001C9C10B5FFF729FF10BD10B5FFF759FF10BD9A
S31508001CAC10B5FFF7A3FF10BD10B5FFF7E9FF10BD80
S31508001CBC10B5FFF773FF002800D110BDFFF7C4FF5E
S31508001CCCFBE70000054BDB699B0604D5034B5B6AF7
S31508001CDC0370012070470020FCE7C0460044004012
S31508001CEC10B5084B986200F0CBF80A300400054B87
S31508001CFCDB691B0605D400F080F900F0C1F8A04298
S31508001D0CF5D910BD0044004030B589B00C4C236899
S31508001D1C0125AB432360E1231B02019300230293A5
S31508001D2C039304930C220592069307930093694632
S31508001D3C2000FFF79DFC23682B43236009B030BDB8
S31508001D4C0044004070B506000D00402904D8280050
S31508001D5CFFF7C6FF00240BE07621074800F09CF835
S31508001D6CF5E700F04AF9305DFFF7BAFF0134A4B283
S31508001D7CABB2A342F5D870BDD425000870B50600E1
S31508001D8C0D00264B1C78002C17D12548FFF79AFF17
S31508001D9C012801D0200070BD214B1B78013BDBB21A
S31508001DAC3F2BF7D800F06CF81E4B18601E4B002220
S31508001DBC1A701A4B01321A70ECE71B4B1B7801335D
S31508001DCC1748C018FFF77EFF0400012817D1164BD9
S31508001DDC1A780132D2B21A70114B1B789A4201D07A
S31508001DEC0024D7E792B20E4901313000FFF700FD07
S31508001DFC0A4B00221A700C4B1B782B70CAE700F0A2
S31508001E0C3FF8084B1B686433984204D9034B0022ED
S31508001E1C1A700024BEE70024BCE7C04695040020CF
S31508001E2C540400209804002096040020024B00223B
S31508001E3C1A605A609A60704710E000E010B5FFF718
S31508001E4CF5FF054B054A5A6000229A600521196070
S31508001E5C034B1A6010BDC04610E000E0FFF9000005
S31508001E6C9C040020044B1B68DB0303D5034A136848
S31508001E7C013313607047C04610E000E09C04002054
S31508001E8C10B5FFF7EFFF014B186810BD9C04002036
S31508001E9C10B5FFF7F5FF10BD10B500F0AEF8FCE76E
S31508001EAC10B500F09FF8012803D00B4B1B78012BBB
S31508001EBC00D010BDFFF7E4FF084B1B68084A1268F0
S31508001ECC9B18F533FF339842F3D3034B00221A7051
S31508001EDCFFF76CFCEDE7C046A4040020A004002024
S31508001EECA804002010B5054B1B78012B00D010BD9B
S31508001EFCFFF7C6FF024B1860F9E7C046A40400209A
S31508001F0CA804002010B5044B01221A70FFF7EAFF4B
S31508001F1CFFF7C6FF10BDC046A404002010B5FFF796
S31508001F2C41FC00F066F8FFF789FFFFF7ADFE00F0FD
S31508001F3C0DF8FFF7E7FF10BD10B500F05EF8FFF7D8
S31508001F4C91FF00F00FF8FFF7ABFF10BD10B500F0CE
S31508001F5CCFF9FFF7D9FE024B00221A7010BDC04606
S31508001F6C0C00002000B583B06B46D91D0748FFF757
S31508001F7C05FF012801D003B000BD054B00221A70DD
S31508001F8C6B46D979014800F0D3F9F4E7AC04002084
S31508001F9C0C0000207047000010B5054B1B78002B71
S31508001FAC02D000F0BDF910BDC9B2FFF7CBFEF8E7B9
S31508001FBC0C000020044B1B78013BDBB2022B01D929
S31508001FCC402000E0002070470C000020044B1B78D2
S31508001FDC013BDBB2022B01D9402000E00020704700
S31508001FEC0C00002010B500F091F9002800D0012053
S31508001FFC10BD10B5FEF728F910BD10B5FEF729F976
S3150800200C10BD0000014B00225A707047EC040020EA
S3150800201C034BFE22DA701871BA3A022199527047AC
S3150800202CEC04002010B5054C00232370FFF7EAFFDB
S3150800203CFF23E370BB3B0122E25210BDEC040020E7
S3150800204C064BFF22DA7000221A71597859719A7167
S3150800205CDA711A724432062199527047EC04002040
S3150800206C10B50020FFF7D4FF10BD0000094BFF2266
S3150800207CDA70094A9A6400221A715A719A71072100
S3150800208CD9710021197259729972442208319952E0
S3150800209C7047C046EC040020EC260008044BFF22CF
S315080020ACDA7042689A644422012199527047C046F4
S315080020BCEC04002010B53120FFF7AAFF10BD000074
S315080020CC70B5084CFF23E370002525716571FFF781
S315080020DC71FFA071E5712572657244230722E252DD
S315080020EC70BDC046EC04002070B5FFF78BFF0D4C95
S315080020FC01252570FF23E370EF3B237100236371E1
S3150800210CFFF758FFA071FFF761FFE071FFF75EFF5D
S3150800211C000A20726572A57244230822E252FFF760
S3150800212CB3FD70BDEC04002070B505004478FFF7CC
S3150800213C41FF0138844211DC6A780A4C201DA16CD7
S3150800214CFFF756FBFF23E3706B78A26C9446634447
S3150800215CA3646B7801334422A35270BD2220FFF787
S3150800216C57FFFAE7EC04002070B504004578FFF732
S3150800217C21FF0138854212DC61680B4DA96462782F
S3150800218C281DFFF735FBFF23EB706378AA6C944682
S3150800219C6344AB64637801334422AB5270BD22208E
S315080021ACFFF736FFFAE7C046EC040020F8B5050041
S315080021BC1700002406E02B781C19E4B20135FFF74A
S315080021CC1CFF31004E1E0029F5D13C600120F8BDDC
S315080021DC10B5084CFF23E370E21D4168A06CFFF7AD
S315080021ECE5FF207100236371A37144330822E25280
S315080021FC10BDC046EC04002070B504000E4B9D6C57
S3150800220CFFF7D8FE411E621C2800FFF741FD002887
S3150800221C0DD0094CFF23E370FFF7CCFE0138A36CF5
S3150800222C9C466044A06444230122E25270BD3130BE
S3150800223CFFF7EEFEFAE7C046EC04002070B5040082
S3150800224C4578FFF7B7FE0238854210DC134BFF22A0
S3150800225CDA70BB3A01219952617800290BD1FFF744
S3150800226C27FD002806D13130FFF7D2FE02E02220E6
S3150800227CFFF7CEFE70BD094B986CA21CFFF708FD44
S3150800228C002806D06378054A916C8C46634493649F
S3150800229CF0E73130FFF7BCFEECE7C046EC04002053
S315080022AC10B5094B9B6C41681800FFF7F5FC002824
S315080022BC06D0054BFF22DA70BB3A0121995210BDA4
S315080022CC3130FFF7A5FEFAE7EC04002010B5FFF74E
S315080022DC6DFA034BFF22DA70BB3A0121995210BDF5
S315080022ECEC04002010B589B2FFF756FE10BD0000AD
S315080022FC054B00221A709A6443215A5401315A52DA
S3150800230C9A705A707047C046EC040020034B1B7831
S3150800231C002B01D0012070470020FCE7EC040020BC
S3150800232C024A43230021D1547047C046EC040020CE
S3150800233C10B50378FF2B04D0294A1278012A14D039
S3150800234C10BDFFF7D1FE264A4323D35C012B42D09E
S3150800235C234A4423D15E0029F2DD100043230122CF
S3150800236CC2540330FFF7BEFFEAE73733DAB2352A31
S3150800237C2DD893001B4AD3589F46FFF7D5FEE2E7A4
S3150800238CFFF7F2FEDFE7FFF789FEDCE7FFF720FF32
S3150800239CD9E7FFF76BFED6E7FFF762FED3E7FFF741
S315080023AC4FFED0E7FFF73EFECDE7FFF725FFCAE75E
S315080023BCFFF744FFC7E7FFF783FEC4E7FFF770FF95
S315080023CCC1E7FFF783FFBEE7FFF774FEBBE72020E4
S315080023DCFFF71EFEB7E71020FFF71AFEB8E7C04650
S315080023ECEC0400201426000870B500260C4D0D4C84
S315080023FC641BA410A64209D1002600F021F80A4D48
S3150800240C0A4C641BA410A64205D170BDB300EB5848
S3150800241C98470136EEE7B300EB5898470136F2E7D2
S3150800242CF4260008F4260008F4260008F826000806
S3150800243C03001218934200D1704719700133F9E75B
S3150800244CF8B5C046F8BC08BC9E467047F8B5C046F9
S30D0800245CF8BC08BC9E46704757
S3150800246410B50C4A54698023DB0223435361EFF306
S31508002474108472B6002303E004C904C00133DBB236
S315080024843F2BF9D9034B1B69DB03FBD484F3108870
S30D0800249410BDC04600200240FD
S3150800249C0000000000000000000000000000000022
S315080024AC0000000000000000000000000000000012
S315080024BC01000000020000000300000004000000F8
S315080024CC06000000070000000800000009000000D4
S315080024DC00000000000000000000000000000000E2
S315080024EC01000000020000000300000004000000C8
S315080024FC01000000020000000400000006000000B5
S3150800250C080000000A0000000C0000001000000083
S3150800251C20000000400000008000000000010000C0
S3150800252C002800080008000005000000003000081C
S3150800253C000800000600000000380008000800002B
S3150800254C0700000000400008000800000800000012
S3150800255C00480008000800000900000000500008A8
S3150800256C000800000A0000000058000800080000D7
S3150800257C0B00000000600008000800000C000000BA
S3150800258C00680008000800000D0000000070000834
S3150800259C000800000E000000007800080008000083
S315080025AC0F000000008000080080000010000000EA
S315080025BC00000108008000001100000000800108DE
S315080025CC0080000012000000433A2F576F726B2FE1
S315080025DC736F6674776172652F4F70656E424C54D3
S315080025EC2F5461726765742F536F757263652F412B
S315080025FC524D434D305F53544D333247302F72731F
S3150800260C3233322E63000000B6230008DA230008A2
S3150800261CDA230008D4230008DA230008DA23000892
S3150800262CCE230008BC230008C8230008C2230008D0
S3150800263CDA230008DA230008DA230008DA2300086C
S3150800264CDA230008DA230008DA230008DA2300085C
S3150800265CDA230008DA230008DA230008DA2300084C
S3150800266CDA230008DA230008DA230008DA2300083C
S3150800267CDA230008DA230008DA230008DA2300082C
S3150800268CDA230008DA230008DA230008DA2300081C
S3150800269CDA230008DA230008DA230008DA2300080C
S315080026ACDA230008DA230008DA230008DA230008FC
S315080026BC982300088C230008862300089223000818
S315080026CCDA230008DA230008DA2300089E23000818
S315080026DCDA230008A4230008AA230008B02300085C
S30D080026EC4F70656E424C540064
S309080026F4E5000008E7
S309080026F8BD0000080B
S315080026FC0024F4000100000004000000040000009F
S7050800056984
